:020000020000FC
:1000000000C00FEF0DBF00E10EBF0FEF04BB0FEFFD
:1000100005BB01E001BB01E002BB0C94B500442725
:100020000CE00093700000E00093710004EC00937A
:100030007400789404EA009374000091740007FF40
:10004000FCCF00917100087F083011F00C948B00F8
:1000500004E00093740000EE0093730004E8009342
:1000600074000091740007FFFCCF00917100087FBD
:10007000083111F00C948D0004E00093740000E04E
:100080000093730004E8009374000091740007FF6C
:10009000FCCF00917100087F083211F00C948F00A2
:1000A00004E900937400009174000071E1F704EA20
:1000B000009374000091740007FFFCCF0091710061
:1000C000087F083011F00C94990004E0009374004C
:1000D00001EE0093730004EC00937400009174002F
:1000E00007FFFCCF00917100087F003421F504E880
:1000F000009374000091740007FFFCCF0091710021
:10010000087F0835E1F42091730004E9009374003E
:10011000209525BBFDCF41E014C042E012C043E072
:1001200010C044E00EC045E00CC046E00AC047E005
:1001300008C048E006C049E004C04AE002C04BE005
:1001400000C010917100142B109515BBFFCFBF9309
:10015000AF931F93BFEFAFEF1FEF1197F1F71A9512
:10016000E1F71F91AF91BF91089550E055BBFFCFCC
:020170000895F0
:00000001FF
